:100000000C9437010C946F010C946F010C946F01E8
:100010000C946F010C946F010C946F010C946F01A0
:100020000C946F010C946F010C94DA1C0C94AC1DB1
:100030000C9411180C946F010C946F010C946F01C7
:100040000C946F010C946F010C946F010C946F0170
:100050000C946F010C946E180C946F010C946F014A
:100060000C946F010C946F010C946F010C946F0150
:100070000C946F010C946F010C946F010C946F0140
:100080000C946F010C946F010C946F010C946F0130
:100090000C9491020C946F010C946F010C946F01FD
:1000A0000C946F010C946F010C946F0195059505EC
:1000B000C105C105290647065F075F075206EB0623
:1000C000FC06FC06191E401E381F401E381F8C1EE1
:1000D000AF1E381F061F151F49004A004B004C0079
:1000E0004D004E0000000000000000005200000023
:1000F000500051004F00160344004300300031000F
:1001000020004100720072006F00770000001603AB
:100110004D0065006300680062006F0061007200BE
:100120006400730000000403090409023B0002019B
:1001300000A0FA09040000010301010009211101D6
:1001400000012240000705810308000109040100A5
:10015000010300000009211101000122B60007057A
:1001600082032000011201000200000008688912C9
:100170001001000102000105010902A10185020927
:1001800001A1000509190129081500250195087527
:100190000181020501093009311581257F9502751C
:1001A00008810609381581257F95017508810605A6
:1001B0000C0A38021581257F950175088106C0C09B
:1001C00005010980A101850319012AB7001501263F
:1001D000B700950175108100C0050C0901A10185CA
:1001E0000419012AA002150126A0029501751081AB
:1001F00000C005010906A1018506050719E029E7E8
:10020000150025019508750181020507190029EFE0
:100210001500250195F075018102050819012905D0
:10022000950575019102950175039101C0050109BC
:1002300006A101050719E029E715002501950875B4
:100240000181029501750881010507190029FF1533
:100250000026FF009506750881000508190129058B
:10026000950575019102950175039101C000112456
:100270001FBECFEFDAE0DEBFCDBF04B603FE18C06D
:100280008091A2029091A302A091A402B091A50234
:100290008730904BA740B04B59F41092A2021092B5
:1002A000A3021092A4021092A502E0E0F8E30995DF
:1002B00011E0A0E0B1E0E6EDFFE302C005900D9291
:1002C000A438B107D9F722E0A4E8B1E001C01D923B
:1002D000A23AB207E1F70E94F7110C94E91F0C94BF
:1002E000000008950C9471010C9472010C9471013A
:1002F000CF93DF93ACE1B1E041E251E061E070E027
:100300008D91E82FE295EF70F0E021A18F70EB0165
:1003100002C0CC0FDD1F8A95E2F7CE019C2F90958D
:10032000922391A392A1892B82A34A175B0741F7DD
:10033000A9E1B1E04CE151E061E070E08D91E82F7E
:10034000E295EF70F0E021A18F70EB0102C0CC0FBD
:10035000DD1F8A95E2F7CE019C2F9095922391A301
:1003600092A1892B82A34A175B0741F7EBE8F1E0E2
:10037000A6E8B1E080E991E011921D928E179F07E7
:10038000D9F7DF91CF910C9440034F925F926F9217
:100390007F928F929F92AF92BF92CF92DF92EF9215
:1003A000FF920F931F93CF93DF932CE1C22E21E096
:1003B000D22E06E811E0E801EE24E394F12CBB24F0
:1003C000B394BE0198801882D6018D916D01E82FFB
:1003D000E295EF70F0E021A18F70A70102C0440FF9
:1003E000551F8A95E2F7CA01242B21A322A1A42E2E
:1003F000A0942A2122A350EA5A95F1F799E1492EB7
:1004000091E0592E20E030E0D2018D902D01482D51
:1004100042954F7050E0DA0190966C907880582D9C
:100420005F70D70102C0AA0FBB1F5A95E2F7AD015A
:10043000562D542341F45E2D022E01C0550F0A940F
:10044000EAF7452F01C040E0472948832F5F3F4F1F
:1004500023303105C9F691A1A922A1A292A1892B2D
:1004600082A32196FB018081981641F0B092900101
:100470000E9447189093920180939101F1E0CB384C
:10048000DF0709F09ECF809190018823A1F0809131
:100490009101909192010E945F18069760F0EBE83D
:1004A000F1E0D8018D918D018193B1E00B381B07EC
:1004B000C1F71092900185E580937202EBE8F1E0BC
:1004C00082E090E02191DC01AF58BD4F2C93019662
:1004D00087309105B9F70E94420381E0DF91CF9107
:1004E0001F910F91FF90EF90DF90CF90BF90AF9052
:1004F0009F908F907F906F905F904F900895E82F1E
:10050000F0E0E557FE4F80810895089580E40E9451
:100510008B02789408958093BA0085EC8093BC0098
:1005200008951F920F920FB60F9211248F939F93ED
:10053000EF93FF938091B900887F803869F038F499
:100540008823B1F18036B1F51092930133C0883A17
:1005500009F1883BF9F02EC080919301811111C0FF
:100560008091BB0080939401809194018E3120F0A2
:100570001092940180E001C081E091E0909393019A
:100580001AC0E0919401F0E08091BB00EF58FD4F5C
:10059000808308C0E0919401F0E0EF58FD4F808126
:1005A0008093BB00809194018F5F8093940102C07F
:1005B0001092BC0081E09091BC008295880F880F5A
:1005C000807C9568892B8093BC00FF91EF919F916F
:1005D0008F910F900FBE0F901F90189581E0089596
:1005E00081E008950C94F00208950C94F4021F9396
:1005F000CF93DF9300D000D01F92CDB7DEB74983F1
:100600005A836B833091960189819A81311114C08C
:10061000662359F0222349F00E949C09182F682F65
:1006200089819A810E94450903C00E947009182F90
:1006300069817A81812F04C00E949C0969817A8135
:100640000F900F900F900F900F90DF91CF911F910F
:100650000C94BB10FC01262F408151816281738173
:1006600084810C94F70281E00895CF93DF93EC012D
:1006700060E00E942A03BE01DF91CF910C94F50245
:100680000C9474010C94760108950E94EF070E9467
:1006900044032FEF84E39CE0215080409040E1F739
:1006A00000C000000C9494180F931F93CF93DF9316
:1006B0008C0161E00E942A03EC01B8010E94F20261
:1006C0008823F1F1B801CE010E9479168823C1F187
:1006D000B801CE010E948D14882391F1B801CE019A
:1006E0000E94D515882361F1F8018281882309F1E0
:1006F000CB358DE5D807C1F050F4C115FCE5DF0717
:1007000081F0CF3DDC45A9F40E94D30E19C0CC3551
:10071000EDE5DE0761F0CD35DD4559F40E94160E9A
:1007200008C00E9445030CC00E941F0E02C00E9418
:10073000220EC801DF91CF911F910F910C94EE0210
:1007400080E0DF91CF911F910F9108950E94BB032C
:100750000C940E1808950C94AA0381E008950C944B
:10076000AD030895CF93C82F0E94AB038C2F0E9436
:10077000AF03CF9108950E94D5160C94B2030E9446
:10078000D51690919501891721F0809395010C94CD
:10079000B2030895CF93DF93CDB7DEB72B970FB693
:1007A000F894DEBF0FBECDBF4F83588769877A8725
:1007B0008B8761110E94620D9E012F5F3F4F86E083
:1007C000F90111928A95E9F785E0FE013796D90182
:1007D00001900D928A95E1F789819A814C815D8122
:1007E000452B31F09F3F31F491E08F3F19F403C066
:1007F00091E001C090E090FF09C049815A816B816E
:100800007C818D819E810E94830C05C0C9010E945C
:1008100033038111F2CF2B960FB6F894DEBF0FBED3
:10082000CDBFDF91CF910895FC01808191810E941D
:10083000DE090895CF93882309F4A4C0C82F823815
:10084000C1F40E94D51681FD9DC069E3809102012B
:10085000909103010E94CB170E94840D2FEF81EE2F
:1008600094E0215080409040E1F700C0000069E32F
:1008700019C0833801F50E94D51680FD83C063E559
:1008800080910201909103010E94CB170E94840D78
:100890002FEF81EE94E0215080409040E1F700C0BE
:1008A000000063E580910201909103010E94D61738
:1008B000CF910C94840D8438C1F40E94D51682FD2A
:1008C00061C067E480910201909103010E94CB17FF
:1008D0000E94840D2FEF81EE94E0215080409040E3
:1008E000E1F700C0000067E4DDCF8CEF8C0F813AA8
:1008F000D0F46C2F80910201909103010E944B175C
:10090000882349F06C2F80910201909103010E948D
:10091000D6170E94840D6C2F8091020190910301E3
:100920000E94CB17C5CF80E28C0F883048F4C77087
:1009300081E001C0880FCA95EAF70E94450DB8CF43
:10094000EBE5EC0FE33040F4F0E0E15BFE4F80813B
:1009500090E0CF910C940917E8E5EC0FE73150F4E3
:10096000F0E0EE0FFF1FEF5DFE4F80819181CF9190
:100970000C941F17CD3E30F08C2F0E947C12CF912B
:100980000C944E13CF910895882309F464C08238E3
:1009900079F40E94D51681FF5EC069E3809102015F
:1009A000909103010E94CB170E94840D69E310C04F
:1009B0008338B1F40E94D51680FF4DC063E5809165
:1009C0000201909103010E94CB170E94840D63E500
:1009D00080910201909103010E94D6170C94840D1E
:1009E000843879F40E94D51682FF35C067E480917F
:1009F0000201909103010E94CB170E94840D67E4CD
:100A0000E7CF9CEF980F913A10F4682FE1CF90E276
:100A1000980F983050F4877091E001C0990F8A9533
:100A2000EAF7892F0E944B0DD9CF9BE5980F9330A1
:100A300020F480E090E00C94091798E5980F973126
:100A400020F480E090E00C941F178D3E20F00E946F
:100A5000D7120C944E1308951F93CF93DF93182F42
:100A6000EB010E941A04209741F08FE99FE0019763
:100A7000F1F700C000002197F6CF812FDF91CF91D1
:100A80001F910C94C404893319F060E070E002C037
:100A900060E570E00C942C05882321F00E94450D40
:100AA0000C94840D0895882321F00E944B0D0C9422
:100AB000840D0895CF92DF92EF92FF920F931F93D0
:100AC000CF93DF937C01D62FC72FFC0112810581C4
:100AD00002950F700E943B0D8823B9F01123A9F0F5
:100AE0008C2F807F803421F080E28D0F883068F079
:100AF0008091900282FD09C082E00E94E40D0E9474
:100B00003B0D91E0D82ED92601C0D12CCC2EC29419
:100B10008FE0C8228C2D90E08C30910508F0CFC179
:100B2000FC01EA5AFF4F0C94801F8C2F807FCF70FE
:100B3000882311F0C295C07F112399F0CC2309F4CA
:100B4000AAC180E28D0F883010F0D11104C08C2F23
:100B50000E94450D03C08C2F0E94550D0E94840DEC
:100B60009AC18D2F0E94C404CC2309F4A8C180E24D
:100B70008D0F883038F1DD2329F18C2F0E945B0D19
:100B800024C08C2F807FCF70803211F0C295C07F3F
:100B9000DD2319F0D130A1F13DC08091900282FF98
:100BA00017C0112349F0CC2329F08C2F0E94450D4A
:100BB0000E94840D80E070C180E00E94C404CC23B8
:100BC00009F47DC18C2F0E944B0D0E94840D77C1CA
:100BD000112371F0002341F0013031F40E94650DC2
:100BE0008C2B0E946D0D6BC10E94650D8C2B1DC05E
:100BF000002319F0013009F462C10E947A0D25C06A
:100C0000112321F0063008F05AC10EC0053008F05B
:100C100056C11BC0112361F0002331F0F70185811B
:100C200080FF39C18F7085838C2F0E944C0547C18E
:100C3000002359F0D93309F03FC1FFEF07EE13E06D
:100C4000F15000401040E1F735C18C2F0E94530550
:100C500036C18C2F86958695837019F0813061F0AE
:100C60002EC1112321F08D2F9C2F937002C080E0A4
:100C700090E00E9409172BC1112321F08D2F9C2F8A
:100C8000937002C080E090E00E941F1720C18D2F5A
:100C9000112319F00E947C1202C00E94D7120E94F8
:100CA0004E1315C18C2F837009F047C011110BC171
:100CB0002D2F229526952770220F220F6D2F6F70F2
:100CC000862F90E0A0E0B0E0022E04C0880F991FAC
:100CD000AA1FBB1F0A94D2F7D4FF10C04FE050E008
:100CE00060E070E004C0440F551F661F771F2A950F
:100CF000D2F7409550956095709503C040E050E064
:100D0000BA01C695C695C3708A019B01082B192BA1
:100D10002A2B3B2BC901B801C23049F058F4C1302D
:100D200019F00E945B08CFC00E944908CCC00E9405
:100D30006D08C9C00E944708C6C0112319F08C2F46
:100D4000817001C08695882309F4BDC02D2F22959E
:100D500026952770220F220F6D2F6F70862F90E03F
:100D6000A0E0B0E0022E04C0880F991FAA1FBB1F8D
:100D70000A94D2F7D4FF10C04FE050E060E070E07A
:100D800004C0440F551F661F771F2A95D2F7409560
:100D900050956095709503C040E050E0BA01C6954B
:100DA000C695C3708A019B01082B192B2A2B3B2B5C
:100DB000C901B801C23049F058F4C13019F00E949D
:100DC000200981C00E940E097EC00E9432097BC0AA
:100DD0000E94810878C0CF70112339F08C2F0E94B7
:100DE000A7088D2F0E944C056EC08D2F0E945305C1
:100DF0008C2F0E94C80867C0D23F21F128F4D03F51
:100E000041F0D13FC1F043C0D33F19F1D43F79F055
:100E10003EC0112341F0053008F051C08C2F8F7176
:100E20000E94ED084CC0063008F049C0F7CF809111
:100E3000900282FF18C0112339F08C2F8F710E940D
:100E4000A7083DC01123C9F38C2F8F710E94C808D9
:100E500036C0112329F08C2F8F710E9492082FC069
:100E60000E948D082CC0112349F0CF718C2F0E9455
:100E7000A70863E08C2F0E94C90D21C081E00E9469
:100E8000E40D0230E0F082E00E94E40D18C011236E
:100E900031F0002391F28D2F0E941A0410C000231C
:100EA00099F2D93349F41FEF27EE33E01150204077
:100EB0003040E1F700C000008D2F0E94C40488EF8D
:100EC0008C0D843020F40E94D5160E94B203DD20E0
:100ED000C9F00E94370D80FD15C0F70112820E94F3
:100EE000310D0E94A708C7010E94A3070E94310D7F
:100EF000DF91CF911F910F91FF90EF90DF90CF90F6
:100F00000C94C808DF91CF911F910F91FF90EF9043
:100F1000DF90CF9008950F931F93CF93DF93EC0151
:100F2000688179818A810E94E9098C010E944409C3
:100F30000E943508B801CE010E945A05DF91CF9179
:100F40001F910F910895CF93DF93EC0198818981D0
:100F50002B813C81232B31F08F3F31F481E09F3F87
:100F600019F403C081E001C080E080FD1DC0CE0106
:100F70000E945403811110C00E943B0D8823A1F0F0
:100F80008A81882389F08091900282FD0DC082E0E1
:100F9000DF91CF910C94E40DCE010E948B07CE011E
:100FA000DF91CF910C943503DF91CF91089580E0CC
:100FB00090E00E94091780E090E00E941F170E94B5
:100FC000620D0E94840D0E947F140C944E13809138
:100FD0000201909103010E94E1170C94D7070E942F
:100FE000520D0C94E70792959F70963079F010F4AB
:100FF000925001C09A50923068F4803F69F018F422
:10100000883E40F409C0843F29F406C0883E20F0A1
:10101000813F11F080E0089581E00895FC01808116
:1010200091810E94DE090E94F3070895CF93DF9318
:1010300000D000D01F92CDB7DEB70F900F900F9069
:101040000F900F90DF91CF910895CF93DF9300D051
:1010500000D000D0CDB7DEB726960FB6F894DEBF2D
:101060000FBECDBFDF91CF910895089508950C94E0
:1010700036080C9437080E9439086093A5017093D4
:10108000A6018093A7019093A8010C94D7070C9414
:101090003B080F931F930091A5011091A601209189
:1010A000A7013091A801602B712B822B932B1F91EC
:1010B0000F910C943B080F931F930091A501109181
:1010C000A6012091A7013091A801602371238223FA
:1010D00093231F910F910C943B080F931F93009142
:1010E000A5011091A6012091A7013091A8016027C8
:1010F0007127822793271F910F910C943B080C9422
:1011000036080E947F086093A1017093A20180932A
:10111000A3019093A4010C94D70760E070E0CB0189
:101120000C9481080F931F9341E050E060E070E061
:101130008A019B0104C0000F111F221F331F8A95D3
:10114000D2F7C901B8011F910F910C9481080F9338
:101150001F9341E050E060E070E004C0440F551F71
:10116000661F771F8A95D2F78091A1019091A20105
:10117000A091A301B091A4018A019B01082B192B16
:101180002A2B3B2BC901B8011F910F910C948108A8
:101190000F931F9341E050E060E070E004C0440F03
:1011A000551F661F771F8A95D2F740955095609519
:1011B00070958091A1019091A201A091A301B0919D
:1011C000A4018A019B01082319232A233B23C90177
:1011D000B8011F910F910C9481080F931F9341E068
:1011E00050E060E070E004C0440F551F661F771F99
:1011F0008A95D2F78091A1019091A201A091A301BB
:10120000B091A4018A019B01082719272A273B27AF
:10121000C901B8011F910F910C9481080F931F937E
:101220000091A1011091A2012091A3013091A4018C
:10123000602B712B822B932B1F910F910C948108A3
:101240000F931F930091A1011091A2012091A3017E
:101250003091A40160237123822393231F910F9166
:101260000C9481080F931F930091A1011091A2018A
:101270002091A3013091A401602771278227932731
:101280001F910F910C9481080895292F220F920F1E
:10129000890FE82FE695E695E695877051E001C045
:1012A000550F8A95EAF785E0E89FF0011124E95689
:1012B000FE4F20E030E070E04081CB01022E02C002
:1012C000969587950A94E2F7817081958427852306
:1012D000842781932F5F3F4F2530310569F70895AB
:1012E000292F220F920F890F682F669566956695B4
:1012F000982F977085E0689FB001112440E050E07E
:1013000080E0FB01E40FF51FE956FE4F208130E03D
:10131000092E02C0369527950A94E2F721703327EB
:10132000042E01C0220F0A94EAF7822B4F5F5F4F11
:101330004530510531F70895BF92CF92DF92EF9279
:10134000FF920F931F93CF93DF938C01C090A10165
:10135000D090A201E090A301F090A4018091A5019A
:101360009091A601A091A701B091A801C82AD92AFD
:10137000EA2AFB2ACFE1D0E0D701C6010C2E04C037
:10138000B695A795979587950A94D2F780FD04C0E6
:10139000219790F7B12C07C0BC2EB8018C2F0E946A
:1013A000D1100197A9F38B2DDF91CF911F910F9150
:1013B000FF90EF90DF90CF90BF900895CF93DF9391
:1013C000EC010E949C09BE010E94D110DF91CF91D7
:1013D00008951F93CF93DF93EB019091960199238A
:1013E00021F0CB010E94DE0913C0882349F0CB0114
:1013F0000E949C09182F682FCE010E94450904C045
:10140000CB010E947009182FBE01812F0E94D110BC
:10141000DF91CF911F9108951F93CF93DF93C091D8
:10142000A90116E08091AA01C81799F0D0E01C9F8D
:10143000F0011D9FF00D1124E555FE4F40815181B3
:1014400062817381848195810E9425082196C770ED
:10145000E9CFDF91CF911F9108954091DB01509129
:10146000DC016091DD017091DE018091DF019091DE
:10147000E0010C942508EF92FF920F931F93CF93F6
:10148000DF938091E00182958F7009F065C08091B3
:10149000DD01882309F460C08091A901F090AA01C0
:1014A0001091DB010091DC016091DE017091DF01A0
:1014B00091E01F3F09F090E0C0910001D09101013F
:1014C000292F96E0E92E8F1509F446C061157105A4
:1014D00021F00F3F21F030E003C031E001C0322F96
:1014E00090E030FD36C0E89EF001E99EF00D112439
:1014F000DF01A555BE4F11963C911197301329C0BD
:101500003C91311326C012963C911297311121C0A3
:1015100013964D915C911497461B570B4C175D0722
:10152000C0F48091E0018F7080618093E001E0550C
:10153000FE4F80818F70806180838BED91E00E94EF
:10154000A307DF91CF911F910F91FF90EF900C9423
:101550000C0A01968770B7CFDF91CF911F910F9141
:10156000FF90EF9008959F92AF92BF92CF92DF923B
:10157000EF92FF920F931F93CF93DF93CDB7DEB718
:1015800061970FB6F894DEBF0FBECDBF8C0185E02A
:10159000F801DE011D9601900D928A95E1F7D801C0
:1015A0001296EC909091DB01E091DC012091DE013C
:1015B0003091DF012115310531F0EF3F31F481E049
:1015C0009F3F19F403C081E001C080E0B82FB170E3
:1015D0009B2E80FD47C1D8014C9111965C911197CB
:1015E0001396AD90BC9014978BEDC82E81E0D82E49
:1015F000F090DD01B501621B730B20910001309169
:101600000101FF2009F4D9C08091E001621773073E
:1016100008F095C0282F207F09F052C05E1313C038
:10162000491311C0FE2CE1100EC08F7080618093B1
:10163000E0010E942D0AC6010E94A3078091E001EB
:10164000F80185834DC1AB2831F05F3F31F481E073
:101650004F3F19F403C081E001C080E080FD03C06A
:1016600081E08E2502C080E090E0F82FF170FF2E1F
:1016700080FF1CC08091A9012091AA0136E0821749
:1016800009F40BC190E0389FF001399FF00D11244F
:10169000E555FE4F6181561306C06081461303C0B5
:1016A0006281E61203C001968770E9CFFE2CEE201E
:1016B00009F416C18091E00181608093E00154C07B
:1016C0005E1306C0491304C0E11002C0F80199C0BE
:1016D000C8010E940E08882361F1EE2051F120918B
:1016E000E001822F82958F7090E0029774F08091D4
:1016F000DB019091DC0198878F831986BB86AA86CF
:101700002C87CE0107960E94A30786E0F801ABED77
:10171000B1E001900D928A95E1F70E943B0A0E9488
:101720002D0A0AC05E1711F1C8010E940E0881112E
:101730002CC0C8010E94A307FF24F394D1C0282F16
:10174000207F81F77A2DB98AA88A6E2D89890E9417
:1017500016088BED91E00E94A30786E0D6011D924A
:101760008A95E9F70E942D0AF12CBAC04913DCCF03
:10177000E110DACFF8018583C8010E94A30786E053
:10178000D6011D928A95E9F7ABC0EE2091F2209127
:10179000E001822F82958F7090E002970CF4B5CF14
:1017A0008091DB019091DC019A8389831B82BD8249
:1017B000AC822E83CE010196A6CF6217730708F084
:1017C00044C0FE2CEE2009F4B4CF5E1330C04913A0
:1017D0002EC02091E00120FD21C0822F82958F70C4
:1017E000482F50E041155105C9F0F80125834F30CD
:1017F000510541F08F5F982F9295907F822F8F70C7
:10180000892B8583C8010E94A30786E0F801ABED10
:10181000B1E001900D928A95E1F73CC086E0F801B5
:10182000ABEDB1E001900D928A95E1F759C0C80186
:101830000E940E08811169CF8091E0018160809340
:10184000E001C8010E94A3074BC07A2DB98AA88A7B
:101850006E2D89890E94160886E0D6011D928A9510
:10186000E9F718C0EE2009F464CFC8010E940E0801
:10187000F82E882309F45DCF86E0F801ABEDB1E0E6
:1018800001900D928A95E1F78BED91E00E9414048E
:101890000E943B0A0E942D0A23C04D875E878D85DA
:1018A0009E850E94DE09292F22952F70223028F470
:1018B0009F7039F0811105C00BC0243028F49F704F
:1018C00049F4805E883020F0C8010E94A3079F2C55
:1018D000F92C06C0D80115969C91907F91F7F8CF0E
:1018E0008F2D61960FB6F894DEBF0FBECDBFDF918E
:1018F000CF911F910F91FF90EF90DF90CF90BF900D
:10190000AF909F9008951F93CF93DF93CDB7DEB72D
:101910002C970FB6F894DEBF0FBECDBF4F8358870C
:1019200069877A878B879C87CE0107960E94B30AC6
:101930008823D1F09F8188852A853B85232B31F030
:101940008F3F31F481E09F3F19F403C081E001C073
:1019500080E080FD47C04F81588569857A858B85F9
:101960009C850E9425083EC086E0FE013796DE0178
:10197000119601900D928A95E1F7FF81E8856A85BD
:101980007B856115710531F0EF3F31F481E0FF3F58
:1019900019F403C081E001C080E080FD23C02091E4
:1019A000AA0130E0C9010196877099274091A901E9
:1019B00050E084179507F1F1F983EA837D836C8306
:1019C00096E0929FD001939FB00D1124A555BE4F74
:1019D000FE01319601900D929A95E1F78093AA014C
:1019E0000E940C0A16E08091A9019091AA01891722
:1019F00071F1189FC001112485559E4F0E94B30AB2
:101A0000882329F1E091A9011E9FF0011124E555D9
:101A1000FE4F4081518162817381848195810E9452
:101A200025088091A90190E00196877099278093FD
:101A3000A901D9CF0E94EF071092AA011092A90123
:101A4000EBEDF1E086E0DF011D928A95E9F72C9637
:101A50000FB6F894DEBF0FBECDBFDF91CF911F91BF
:101A600008958091010285958595859508958091C9
:101A700001028770089590910102977081E009F446
:101A800080E0089580912402089590912402892B8A
:101A90008093240208958095909124028923809355
:101AA0002402089510922402089590912302892B14
:101AB0008093230208958095909123028923809337
:101AC000230208951092230208958091020208953E
:101AD00008950C94680D0C94690D9091900292FDFC
:101AE00008C090910202981721F0809302020C9492
:101AF0006B0D089580910202882329F01092020252
:101B000080E00C946B0D0895CF93DF93E091020178
:101B1000F0910301809124028083E0910201F09111
:101B20000301908180912302892B8083809102029E
:101B3000882381F0E0910201F09103019081892BCB
:101B4000808380910201909103010E9435178111D9
:101B50000E947A0DC0910201D091030140E250E051
:101B600061EE71E0CE010E949A1F892B69F080E23C
:101B7000FE01A1EEB1E001900D928A95E1F7CE0150
:101B8000DF91CF910C94E116DF91CF9108950C94E1
:101B9000680D9091900292FD10C098E0899F90018D
:101BA0001124262B209301020E94A7088091010294
:101BB0008595859585950C94C70D0C94A708109272
:101BC000010280E00C94C70D2091010280958223D0
:101BD00080930102982F977099F430E0482F082ED7
:101BE000000C550B2417350759F09091900292FD87
:101BF00007C08595859585950E94C8080C94DF0DD2
:101C000008959091900292FB222720F9281769F0FD
:101C100080FB92F99093900280918F0290919002B4
:101C20000E944F0E82E00C94E40D08958091900282
:101C300082FB882780F991E089270C94010E81E0CE
:101C40000C94010E80E00C94010E6FEF7FEF80E0AA
:101C500090E00C94D31F80E090E00E94AF1F21E041
:101C6000893E9E4F09F020E0822F089582E090E0A7
:101C70000C94A71F83E090E00C94A71FCF9384E0FF
:101C800090E00E94A71FC82F82E290E00E94A71F49
:101C90002C2F30E0A901582BCA01CF910895CF9382
:101CA000C92F682F84E090E00E94B51F6C2F82E25C
:101CB00090E0CF910C94B51FAB01BC018FE090E098
:101CC0000C94C71FAB01BC0183E190E00C94C71FCB
:101CD00060E070E0CB010C94620E60E070E0CB013C
:101CE0000E945C0E0C94680E69EE7EEF80E090E03E
:101CF0000E94D31F60E082E090E00E94B51F60E088
:101D000083E090E00E94B51F1092A5011092A601F9
:101D10001092A7011092A80160E084E090E00E9478
:101D2000B51F60E082E290E00E94B51F60E085E0B0
:101D300090E00E94B51F60E086E090E00E94B51F31
:101D40006FEF87E090E00E94B51F40E050E0BA01DD
:101D500088E090E00E94C71F60E08DE090E00E9464
:101D6000B51F40E050E0BA0188E190E00E94C71F33
:101D700060E087E190E00E94B51F40E050E0BA01CA
:101D80008CE190E00E94C71F60E070E080E290E08C
:101D90000E94D31F40E050E0BA0188E190E00E9429
:101DA000C71F0C946D0E0C94740E682F8EE090E09B
:101DB0000C94B51F0E94531860932E0270932F024B
:101DC000809330029093310260932A0270932B0229
:101DD00080932C0290932D02089585B7806885BF6B
:101DE00085B7806885BF089581E008950C94F40E4E
:101DF00008950C94F80E0C94F80E0C94FB0E0C94B1
:101E0000F80E0C94FF0E0E94ED0E8DEA91E10E94F7
:101E1000CB160E9486020C94010F0E94F90E0C94BE
:101E2000F80E0E94C7110C94B1030E943E180E9444
:101E300078010E94110F0C94FD0E8F929F92AF9229
:101E4000BF92CF92DF92EF92FF920F931F93CF93A7
:101E5000DF93CDB7DEB72A970FB6F894DEBF0FBE7B
:101E6000CDBF0E94C501982E81110E94DA0E85E235
:101E7000A82E82E0B82E00E010E0802E802F0E9475
:101E80007F02D82EF501C1905F01C826B1F40F5F23
:101E90001F4F0530110589F78FEF89838A831B82D5
:101EA0000E9447188160782F9D838C8349815A81D5
:101EB0006B818D810E94CA032FC08091320281FD07
:101EC0000E948502E12CFF24F3948C2D8F21F1F0E8
:101ED0000E94F60E882399F0EE828F82DF2081E047
:101EE00009F480E088870E9447188160782F9A87DC
:101EF00089874E815F8168858A850E94CA03F801BF
:101F0000EB5DFD4F8081F826F08206C0E394FF0C64
:101F1000F3E0EF12DACFBBCF81E0911001C080E097
:101F20002A960FB6F894DEBF0FBECDBFDF91CF91DA
:101F30001F910F91FF90EF90DF90CF90BF90AF90E7
:101F40009F908F9008950E941D0F0E946C130C9417
:101F5000BF03CF93DF930E94D610EC01811521E5DA
:101F6000920708F045C0811530E5930708F094C04A
:101F7000883E910528F5803E910508F0F8C0883A22
:101F8000910570F4853A910508F07CC08130910587
:101F900009F475C008F4E8C0049708F0E8C0E4C08C
:101FA0008F3B910508F0E0C0C85AD0E0CC0FDD1F90
:101FB000CE5ADE4F0990D881C02DCE019464D8C08E
:101FC000811540E2940758F4811551E0950708F017
:101FD000CEC08D3E910508F4C7C09065C9C0C1153B
:101FE00080E4D80708F4C0C0DF70CE01906AC0C09A
:101FF000811525E59207A8F4811534E5930708F0CB
:1020000095C0811543E5940708F07BC0811552E522
:10201000950708F061C0D82FCC27CE01816F906A58
:10202000A7C0C11589E5D807A0F4C11528E5D207D6
:1020300008F082C0C11536E5D30708F095C08C2F93
:102040000E946A118F7190E0D82FCC27CE01906248
:102050008FC0C1154AE5D40708F474C0CE0190566C
:102060008115904208F080C08D2F8F710E946A11F7
:10207000DD27D0628F71AE01582BCA0179C081E093
:1020800090E076C0C55AD0E0C058DE4F8881C82F96
:10209000D0E0CE0190646CC074E0969587957A95F7
:1020A000E1F7282F23703C2F337081E090E002C0CD
:1020B000880F991F3A95E2F79C68AC01522B9A0160
:1020C0009C2F9F709695969550E2959FE001112464
:1020D000C9018C2B9D2B4CC08370992721E030E0E7
:1020E00002C0220F331F8A95E2F79C2F9695969592
:1020F00080E2989FE0011124C22BD32BCE019C6873
:1021000037C08370992721E030E002C0220F331FCF
:102110008A95E2F79C2F9695969540E2949FE00170
:102120001124C22BD32BCE019A6822C0D82FCC27E2
:10213000CE01846F906A1CC0DC2FCC27CE01806F4B
:10214000906A16C08C2F8F700E946A1194E0D69509
:10215000C7959A95E1F7CF70D0E0DC2FCC27D069F6
:102160009E01282BC90104C080E090E001C0CE018F
:10217000DF91CF910895272F30E0F901EE0FFF1F77
:102180002E0F3F1FF9019FE0899FE00DF11D1124E3
:10219000E60FF11DEE0FFF1FE852FF4F859194915E
:1021A00008950E94BB100E94A90F089582389105DE
:1021B00069F1B0F48133910509F46DC048F48932B6
:1021C000910509F463C08A32910509F469C0089544
:1021D0008533910509F455C089339105B9F0089507
:1021E000833E910569F138F4803E9105B1F0823E5D
:1021F000910509F10895863E9105A9F1873E910563
:10220000B9F1843E910509F064C023C020918F028A
:1022100020FD4FC021FD4DC0089580918F0280FDAB
:1022200044C08091900280FF44C080918F0284FD61
:1022300042C083EE4DC080918F0282FF38C0F5CF3F
:1022400080918F0282FD33C08091900280FD31C069
:10225000ECCF8091900281FF32C080918F0284FD8B
:102260002AC087EE35C080918F0283FF26C0F5CF4C
:1022700080918F0283FD21C08091900281FD1FC05B
:10228000ECCF80918F0285FD1CC01DC080918F0214
:1022900085FD19C016C080918F0286FD16C017C03B
:1022A00080918F0286FD13C010C089E311C082EEB9
:1022B0000FC080EE0DC080E00BC086EE09C084EE3A
:1022C00007C089E205C085E303C08AE201C081E35B
:1022D00090E0089590918F0292FF0DC0282F2871F1
:1022E000283019F4877F846006C0282F2471243099
:1022F00011F48B7F886093FF0DC0282F287128313F
:1023000019F4877E846106C0282F2471243111F4CA
:102310008B7E88612091900220FF0DC0382F38718C
:10232000383019F4877F816006C0382F3171313021
:1023300011F48E7F886021FF0DC0282F287128316D
:1023400019F4877E816106C0282F2171213111F493
:102350008E7E886194FD877E089580E008950C94B8
:10236000250E0E94C5018FE39CE90197F1F700C09B
:1023700000000E94C50180E00E947F0280FF04C02F
:102380000E94AF110C94941808950C94B1110E94FE
:102390002B0E811102C00E94D30E0E94360E809334
:1023A00032020E943E0E9093900280938F020E9410
:1023B000C5110E943A0E682F70E080E090E00E9404
:1023C00047086091A1017091A2018091A3019091B1
:1023D000A4010C947F080E94611A0E94150F0C94AE
:1023E0006D1A0E94711A0E94A30F0C94721A0E9417
:1023F00010180E94481A0E94030F0E94EB110E94BD
:10240000F1110E940D0FFBCF8091390280FF06C0B1
:102410006091090170E0660F771F26C081FF04C03C
:102420006091090184E005C082FF07C06091090145
:1024300088E0689FB001112417C090913802992359
:10244000D1F060910801961788F72091090188E082
:10245000289F90011124929FA001939F500D112459
:1024600070E0CA010E946C1F6038710540F461156C
:10247000710519F406C068E070E0862F08958FE7B3
:10248000089581E008958091390280FF08C060912D
:10249000050170E0759567957595679521C081FF79
:1024A00006C06091050170E07595679519C082FFBF
:1024B00004C06091050170E010C09091370299232B
:1024C00099F0609104019617A0F780910501899F0A
:1024D000C001112470E00E946C1F6038710540F447
:1024E0006115710519F406C061E070E0862F08954A
:1024F0008FE7089581E008958D3E21F40E94041233
:10250000819504C08E3E29F40E94041280933D02FE
:1025100008958F3E21F40E940412819504C0803FEB
:1025200029F40E94041280933C020895893F19F413
:102530000E94431205C08A3F31F40E9443128195E4
:1025400080933E0208958B3F21F40E9443128195AF
:1025500004C08C3F29F40E94431280933F020895E7
:102560009FE0980F983078F421E030E0A90102C094
:10257000440F551F9A95E2F7CA0190913B02892BAF
:1025800080933B0208958D3F21F480913902816050
:102590000BC08E3F21F480913902826005C08F3FCD
:1025A00029F48091390284608093390208958D3E28
:1025B00039F490913D0297FF35C010923D0259C009
:1025C0008E3E29F490913D021916BCF32BC09091D8
:1025D0003C028F3E29F497FF25C010923C0249C06F
:1025E000803F19F41916CCF31DC090913E02893F2B
:1025F00029F41916BCF410923E023BC08A3F19F42C
:1026000097FF10C0F8CF8B3F39F490913F0297FFAE
:1026100009C010923F022DC08C3F21F490913F02DF
:102620001916BCF39FE0980F983080F421E030E059
:10263000A90102C0440F551F9A95E2F7CA0180957F
:1026400090913B02892380933B0213C08D3F21F47C
:10265000809139028E7F0BC08E3F21F48091390228
:102660008D7F05C08F3F29F4809139028B7F809345
:10267000390280913C02811106C080913D02811196
:1026800002C01092380280913E02811106C08091F2
:102690003F02811102C01092370208950E9447182C
:1026A00020913C02211104C020913D02222321F0FF
:1026B000909336028093350220913E02211104C08E
:1026C00020913F02222321F0909334028093330221
:1026D0008AE392E00C94FB16EF92FF920F931F9304
:1026E000CF93DF9300D000D000D0CDB7DEB786E027
:1026F000EAE3F2E0DE01119601900D928A95E1F78E
:10270000E0903C02F0903D0200913E0210913F02A9
:1027100010923C0210923D0210923E0210923F0233
:10272000E11003C0FF2009F45DC080913502909153
:1027300036020E945F18AC0190913802992339F05B
:1027400020910A0130E02417350758F04BC0209142
:102750000B018AE0289F900111242417350718F0F7
:1027600041C09F3F19F09F5F90933802EE2061F0C7
:102770000E9404121E1414F09FEF01C091E0989F74
:10278000902D112490933C02FF2061F00E940412CE
:102790001F1414F09FEF01C091E0989F902D112419
:1027A00090933D0230913C023323E1F020913D02B1
:1027B0002223C1F045EB3403C0011124992319F001
:1027C00090933C0203C081E080933C0235EB2303ED
:1027D000C0011124992319F090933D0203C081E0B8
:1027E00080933D02011103C0112309F45DC0809163
:1027F0003302909134020E945F18AC01909137022D
:10280000992339F02091060130E02417350758F05C
:102810004BC0209107018AE0289F900111242417C2
:10282000350718F041C09F3F19F09F5F9093370222
:10283000002361F00E944312101614F09FEF01C0B4
:1028400091E0989F902D112490933E02112361F006
:102850000E944312111614F09FEF01C091E0989F5F
:10286000902D112490933F0230913E023323E1F0EA
:1028700020913F022223C1F045EB3403C001112413
:10288000992319F090933E0203C081E080933E02A9
:1028900035EB2303C0011124992319F090933F02D3
:1028A00003C081E080933F0280913C0281110BC004
:1028B00080913D02811107C080913E02811103C0C9
:1028C00080913F0281110E944E13EB82FC820D83A6
:1028D0001E8386E0FE013196AAE3B2E001900D92DC
:1028E0008A95E1F726960FB6F894DEBF0FBECDBFEE
:1028F000DF91CF911F910F91FF90EF900895EAE340
:10290000F2E086E0DF011D928A95E9F71092380225
:1029100010923702109239020895CF93DF93EC01A1
:10292000FB018281882309F43CC1C430FDE5DF0747
:1029300060F4CB3F9CE5D90788F49E0122503C45CA
:102940002431310508F02EC109C0C236EDE5DE079D
:1029500029F0C63AFDE5DF0709F024C10E943E0ECA
:102960009093900280938F02C1318CE5D80709F4CF
:10297000C6C008F042C0C930ECE5DE0709F49BC0D0
:1029800000F5C5308CE5D80709F485C078F4C3306C
:10299000ECE5DE0709F478C008F07AC0C230DC4507
:1029A00009F0F5C080918F028160EFC0C7309CE5CF
:1029B000D90709F478C008F07AC080918F0280614D
:1029C000E4C0CD30FCE5DF0709F487C058F4CB3014
:1029D0009CE5D90709F479C008F07BC080918F028B
:1029E00088606FC0CF30FCE5DF0709F480C008F0D5
:1029F00082C080918F02877FC8C0CE3F9CE5D907F7
:102A000009F471C000F5C531FCE5DF0709F485C0A4
:102A100068F4C3319CE5D90709F475C008F095C086
:102A20000E94EF0780918F028F77AFC0CC3FFCE50B
:102A3000DF07A9F108F054C0CB3FDC4509F0A7C07F
:102A40008091900240C0C230EDE5DE0709F489C0F4
:102A500058F4C1158DE5D80709F45AC008F069C0CB
:102A60008091900282602FC0C236EDE5DE0709F446
:102A70007CC0C63AFDE5DF0709F481C0C330DD45FF
:102A800009F085C080E06EC080918F0282607DC0B9
:102A900080918F0216C080918F02886076C08091ED
:102AA000900282604FC080918F0280626EC08091E0
:102AB0008F0280646AC00E94EF0780918F02806855
:102AC00064C0846062C081603DC080918F028E7F4F
:102AD0005CC080918F028D7F58C080918F0216C09C
:102AE0008091900218C0809190028D7F2BC08091C0
:102AF0008F028F7E4AC080918F028F7D46C0809169
:102B00008F028F7B42C080918F02877F8B7F3DC079
:102B1000809190028D7F8E7F15C080918F0282FB05
:102B2000222720F991E0922790FB82F990FB83F90C
:102B30002CC080919002982F909591708E7F892B58
:102B400090FB81F98093900222C00E94EF07809150
:102B50008F0287FB222720F991E0922790FB87F9CB
:102B600014C081E00E94D50E12C080918F0284FBB8
:102B7000222720F991E0922790FB84F906C08091EA
:102B80008F02982F909590FB80F980938F0280910F
:102B90008F02909190020E944F0E0E94EF0780E0FA
:102BA00001C081E0DF91CF910895CF93DF9386310B
:102BB0009C4541F5EB010E94420D982F8A8120919E
:102BC000020130910301882379F09A7A81E009F4B7
:102BD00080E080934002911102C069E201C065E388
:102BE000C9010E94CB170AC080914002811102C026
:102BF00069E201C065E3C9010E94D6170E94840DF5
:102C000080E001C081E0DF91CF9108950F931F9381
:102C1000CF93DF93C42FD22FFC0182818823C9F088
:102C2000409343020E9447189093420280934102CE
:102C300080E28C0F883008F057C0C77081E001C077
:102C4000880FCA95EAF7DF91CF911F910F910C94ED
:102C50004C0580914302481330C08091410290910D
:102C600042020E945F18883C910538F510E21D0F62
:102C7000CD17B9F080E28C0F883040F4C77081E046
:102C800001C0880FCA95EAF70E945305183028F54D
:102C900081E09D2F977001C0880F9A95EAF70E94F6
:102CA0004C05802F0E9443051830F0F4D77081E066
:102CB00001C0880FDA95EAF70AC080E28C0F8830ED
:102CC00098F4C77081E001C0880FCA95EAF7DF91D8
:102CD000CF911F910F910C945305802FDF91CF91CD
:102CE0001F910F910C944305DF91CF911F910F918C
:102CF00008950F939C01CB01243F4CE5340731F13B
:102D000088F4293DFCE53F07D9F02A3D4CE534071E
:102D100079F1283D3C45A9F506E221EE41EE68ED4A
:102D20007CE52BC0263FFCE53F07E1F0A8F0273FFC
:102D30003C4539F507E225EE46EE67EF7CE51DC020
:102D400007E225EE45EE69ED7CE517C006E221EECF
:102D500040EE64EF7CE511C007E225EE44EE65EF3E
:102D60007CE50BC006E221EE42EE66EF7CE505C095
:102D700008E221E045EE6AED7CE50E94061680E05F
:102D800008C0FC018281882319F01092430201C01F
:102D900081E00F91089590938501809384010895B7
:102DA00090934902809348020895E0914802F0917F
:102DB0004902309721F00190F081E02D099480E0E4
:102DC0000895E0914802F0914902309799F02091DE
:102DD0001801222359F020918F0227FF07C0DC0140
:102DE0002C9111962C93119726E02C930280F3815D
:102DF000E02D09940895E0914802F091490230973E
:102E000039F022E0DC012C930480F581E02D099457
:102E1000089520914602309147022817390771F032
:102E20009093470280934602E0914802F091490254
:102E3000309721F00680F781E02D099408952091C4
:102E40004402309145022817390771F090934502EA
:102E500080934402E0914802F0914902309721F0BA
:102E60000084F185E02D09940895FC01329680914B
:102E70001801882331F080918F0287FF02C09EE104
:102E800001C096E080E0915028F021912223D9F3EF
:102E90008F5FF9CF0895662351F120911801222305
:102EA000E9F020918F0227FF19C0462F46954695DD
:102EB00046954E31E0F4677021E030E002C0220F09
:102EC000331F6A95E2F7FC01E40FF11D828190E067
:102ED0002823392381E0232B69F409C0FC013296B1
:102EE00008962191621729F0E817F907D1F780E0D9
:102EF000089581E008959C01FC0132969FEF80E0E7
:102F00004191461789F09F3F19F4411101C0982F54
:102F10008F5F8630A9F79F3F39F0F901E90FF11D66
:102F200097FDFA956283089508959C012A5F3F4FAB
:102F3000FC014281461301C0128201968217930759
:102F4000B9F70895262F2695269526952E3168F4F3
:102F5000FC01E20FF11D677021E030E001C0220F9B
:102F60006A95EAF78281282B22830895262F2695D9
:102F7000269526952E3170F4FC01E20FF11D677045
:102F800021E030E001C0220F6A95EAF720958281A6
:102F900028232283089520911801222329F02091CB
:102FA0008F0227FD0C94A2170C947B172091180117
:102FB000222329F020918F0227FD0C94B6170C9440
:102FC000951720911801FC013296222331F080914F
:102FD0008F0287FF02C08EE101C086E0DF011D92F3
:102FE0008A95E9F7089508950C94F31783E0809388
:102FF0004A020C94F417811102C081E001C082E002
:1030000080934A020C94F4170C94FB1781E0809390
:103010004A020C94F4170C94061808950C940D1899
:1030200008951F920F920FB60F9211248F939F93C2
:10303000AF93BF9380914B02811113C08091910295
:1030400090919202A0919302B09194024196A11D99
:10305000B11D8093910290939202A0939302B0933A
:103060009402BF91AF919F918F910F900FBE0F90DF
:103070001F9018950E94EF070C94A60382E084BD70
:1030800093E095BD9AEF97BD80936E0008952FB79A
:10309000F8948091910290919202A0919302B09144
:1030A00094022FBF08952FB7F89460919102709108
:1030B000920280919302909194022FBF08959C01F7
:1030C0004FB7F8948091910290919202A09193024F
:1030D000B09194024FBF821B930B089578941F9276
:1030E0000F920FB60F9211248F939F93AF93BF93BC
:1030F0008091910290919202A0919302B0919402DA
:103100000196A11DB11D8093910290939202A0930C
:103110009302B0939402BF91AF919F918F910F90C2
:103120000FBE0F901F90189581E08093E00080E221
:103130008093D8001092C9008FE19EE40197F1F7C7
:1031400000C0000087E090EBDC018093A202909326
:10315000A302A093A402B093A5029CE088E10FB65D
:10316000F894A895809360000FBE90936000FFCF05
:1031700080916F020895089522E02093E9002FEFD7
:103180003091E800215035FD06C035ED3A95F1F754
:1031900000002111F5CF2091E80025FF0BC040E091
:1031A00050E066E070E00E94CE1A8091E8008E77D1
:1031B0008093E8000895CF93DF9320911801222394
:1031C00039F020918F0227FF03C060E222E002C0A5
:1031D00068E021E02093E9002FEF3091E8002150D2
:1031E00035FD06C035ED3A95F1F700002111F5CF18
:1031F0002091E80025FF1DC0EC018091180181118C
:1032000005C040E050E068E070E003C070E040E0DE
:1032100050E0CE010E94CE1A8091E8008E77809314
:10322000E80080E2FE01AFE4B2E001900D928A95E1
:10323000E1F7DF91CF91089580934C0270934E0295
:1032400060934D0280919902843001F582E0809371
:10325000E9008FEF9091E800815095FD06C095ED53
:103260009A95F1F700008111F5CF8091E80085FF74
:103270000DC040E050E063E070E08CE492E00E941A
:10328000CE1A8091E8008E778093E8000895BC0103
:1032900084E00C941C19BC0183E00C941C198091EF
:1032A0009802811109C00E945F1C0E94BC1C809181
:1032B000E20084608093E2000895109298020895DD
:1032C0000C940B186091950281E0611101C080E0BF
:1032D0000C94F6170E943A189091990281E094306C
:1032E00009F080E0609195020C94FB1742E061ECDC
:1032F00081E00E94D81B42E261EC82E00E94D81B70
:103300009091990281E0943009F080E060919502FB
:103310000C94041880919B02833009F461C030F44E
:10332000813071F0823009F49AC008958A3009F42E
:1033300086C08B3009F46CC0893009F0A8C020C069
:1033400080919A02813A09F0A2C08091E800877FBB
:103350008093E80080919E0290919F02892B21F436
:1033600060E28FE492E003C060E080E090E070E013
:103370000E94191B8091E8008B778093E8000895E4
:1033800080919A02813209F082C080919E029091D0
:103390009F02029708F07BC08091E800877F8093AE
:1033A000E8008091E80082FD05C0809199028111BA
:1033B000F8CF6DC02091F3008091F20090E0922B45
:1033C000029731F48091F100813011F0863021F4C0
:1033D0008091F10080936F028091E8008B7753C059
:1033E00080919A02813A09F052C080919E02909198
:1033F0009F02892B09F04BC08091E800877F809362
:10340000E8008091E80080FFFCCF8091180136C071
:1034100080919A028132D9F580919E0290919F020B
:10342000892BA9F58091E800877F8093E8000E94AE
:103430000D1C80919C02809318010C94EF078091E1
:103440009A02813221F58091E800877F8093E8001D
:103450000E940D1C80919D028093700208958091BE
:103460009A02813AA1F48091E800877F8093E80076
:103470008091E80080FFFCCF809170028093F10082
:103480008091E8008E778093E8000C940D1C0895DD
:1034900084B7877F84BF0FB6F894A89580916000A9
:1034A000886180936000109260000FBE90E080E819
:1034B0000FB6F89480936100909361000FBE0C9456
:1034C00006180E945F1C0E94BC1CE2EEF0E08081A6
:1034D0008460808378940C94511F8CE091E00C946C
:1034E000D016089508950C94751A292F3327233088
:1034F0003105C9F060F42130310581F02230310509
:1035000009F044C08BE390E02AE231E043C021326D
:103510003105E1F02232310549F138C082E190E015
:1035200025E631E037C099278130910549F028F030
:10353000029761F5E6EFF0E005C0E6E2F1E002C0D7
:10354000EEE0F1E0849190E09F0124C061157105E7
:1035500041F061307105D1F489E090E025E531E07A
:1035600019C089E090E02CE331E014C061157105C9
:1035700041F06130710551F486EB90E027E731E0CE
:1035800009C080E490E02DE232E004C080E090E0E9
:1035900020E030E0FA01318320830895CF92DF925A
:1035A000EF92FF920F931F93CF93DF93EC018B0168
:1035B0007A010E942C1C811133C0E114F10439F00E
:1035C000F70180819181081B190BC80FD91FC12CED
:1035D000D12C0115110519F18091E80085FD16C067
:1035E0008091E8008E778093E800E114F10449F0BF
:1035F000F70180819181C80ED91ED182C08285E0F9
:103600000FC00E942C1C882321F30AC0899180934B
:10361000F10001501109FFEFCF1ADF0ADACF80E085
:10362000DF91CF911F910F91FF90EF90DF90CF909E
:1036300008952091A0023091A1022617370748F083
:103640006115710539F42091E8002E772093E80088
:1036500001C0B901FC0120E06115710579F180918B
:1036600099028823F1F18530F1F18091E80083FD22
:103670003CC08091E80082FD2EC08091E80080FF70
:10368000EBCF2091F3008091F20090E0922B611536
:10369000710551F08830910538F421912093F100A3
:1036A000615071090196F3CF21E0089709F020E0FD
:1036B0008091E8008E778093E800CECF2111CFCFA4
:1036C0000AC080919902882361F0853061F0809171
:1036D000E80083FD0AC08091E80082FFF2CF80E01D
:1036E000089582E0089583E0089581E0089520918F
:1036F000A0023091A1022617370748F06115710525
:1037000039F42091E8002E772093E80001C0B90138
:10371000FC0120E06115710591F1809199028823E7
:1037200009F440C0853009F43FC08091E80083FD72
:103730003DC08091E80082FD2FC08091E80080FFAD
:10374000E9CF2091F3008091F20090E0922B611577
:10375000710559F08830910540F424912093F100CF
:103760003196615071090196F2CF21E0089709F076
:1037700020E08091E8008E778093E800CBCF211184
:10378000CCCF0AC080919902882361F0853061F026
:103790008091E80083FD0AC08091E80082FFF2CFAB
:1037A00080E0089582E0089583E0089581E008951F
:1037B000982F973068F59093E900981739F0709139
:1037C000EC002091ED005091F00003C0242F762FE3
:1037D00050E021FD02C09F5FECCF3091EB003E7FB7
:1037E0003093EB003091ED003D7F3093ED00309150
:1037F000EB0031603093EB007093EC002093ED0010
:103800005093F0002091EE0027FDE5CF80E0089571
:103810008F708093E90081E0089580919A0287FF7C
:1038200011C08091E80082FD05C08091990281114C
:10383000F8CF11C08091E8008B770BC0809199027E
:10384000882349F08091E80080FFF8CF8091E8005C
:103850008E778093E80008952091E4003091E50090
:1038600095E64091EC00842F817040FF23C0809149
:10387000E80080FD1DC080919902882399F0853071
:1038800099F08091EB0085FD11C04091E4005091CA
:10389000E5002417350729F3915011F09A01E1CF83
:1038A00084E0089582E0089583E0089581E008951A
:1038B00080E008954091E80042FFDDCF08950E9426
:1038C000CD1C0E94D51CE0EEF0E0808181608083F9
:1038D000E8EDF0E080818F77808319BCA7EDB0E040
:1038E0008C918E7F8C9380818F7E80831092980242
:1038F00008950F931F93CF93DF930E94CD1C0E94D6
:10390000D51CC8EDD0E088818F7788838881806856
:10391000888388818F7D888319BC109299021092C8
:103920009502109297021092960200EE10E0F801B4
:1039300080818B7F808388818160888342E060E022
:1039400080E00E94D81BE1EEF0E080818E7F8083D2
:10395000E2EEF0E0808181608083808188608083F6
:10396000F80180818E7F8083888180618883DF91E8
:10397000CF911F910F910895E8EDF0E080818F7E47
:103980008083E7EDF0E080818160808384E082BF06
:1039900081E0809398020C94791CE8EDF0E080813E
:1039A0008E7F80831092E20008951092DA001092C8
:1039B000E10008951F920F920FB60F9211242F93DA
:1039C0003F934F935F936F937F938F939F93AF93A7
:1039D000BF93EF93FF938091E10082FF0BC0809132
:1039E000E20082FF07C08091E1008B7F8093E100BD
:1039F0000E94501F8091DA0080FF1FC08091D80084
:103A000080FF1BC08091DA008E7F8093DA00809166
:103A1000D90080FF0DC080E189BD82E189BD09B474
:103A200000FEFDCF81E0809399020E944F1905C0EE
:103A300019BC109299020E945D198091E10080FFEB
:103A400019C08091E20080FF15C08091E2008E7F56
:103A50008093E2008091E20080618093E200809197
:103A6000D80080628093D80019BC85E080939902C9
:103A70000E9462198091E10084FF30C08091E200D1
:103A800084FF2CC080E189BD82E189BD09B400FEBC
:103A9000FDCF8091D8008F7D8093D8008091E10088
:103AA0008F7E8093E1008091E2008F7E8093E20020
:103AB0008091E20081608093E200809195028823EA
:103AC00011F084E007C08091E30087FD02C081E02F
:103AD00001C083E0809399020E946A198091E100FD
:103AE00083FF29C08091E20083FF25C08091E1001F
:103AF000877F8093E10082E0809399021092950283
:103B00008091E1008E7F8093E1008091E2008E7FC2
:103B10008093E2008091E20080618093E20042E0C5
:103B200060E080E00E94D81B8091F0008860809364
:103B3000F0000E946019FF91EF91BF91AF919F91AA
:103B40008F917F916F915F914F913F912F910F9046
:103B50000FBE0F901F9018951F920F920FB60F92E5
:103B600011242F933F934F935F936F937F938F9382
:103B70009F93AF93BF93CF93DF93EF93FF93C09146
:103B8000E900CF708091EC00D82FD17080FDD0E893
:103B90001092E9008091F000877F8093F000789484
:103BA0000E94F01D1092E9008091F00088608093DF
:103BB000F000CD2BCF70C093E900FF91EF91DF9122
:103BC000CF91BF91AF919F918F917F916F915F91B5
:103BD0004F913F912F910F900FBE0F901F9018950E
:103BE0001F93CF93DF93CDB7DEB7AA970FB6F894A4
:103BF000DEBF0FBECDBFEAE9F2E08091F100819314
:103C000022E0E23AF207C9F70E948A198091E8009F
:103C100083FF2EC180919A0290919B02492F50E020
:103C20004A30510508F024C1FA01EE59FF4F0C94B7
:103C3000801F803821F0823809F01AC108C08091B5
:103C4000960290919702992389F082600FC080912B
:103C50009E028F70873008F00BC18093E90080913D
:103C6000EB0085FB882780F91092E9009091E8002D
:103C7000977F9093E8008093F1001092F100D1C0FB
:103C8000282F2D7F09F0F4C0882319F0823061F0CD
:103C9000EFC080919C02813009F0EAC0933009F0B6
:103CA00080E0809397022EC080919C0281112AC0EF
:103CB00080919E028F702FEF280F263008F0D8C019
:103CC0008093E9002091EB0020FF1CC0933021F489
:103CD0008091EB00806214C09091EB009061909312
:103CE000EB0021E030E0A90102C0440F551F8A9586
:103CF000E2F74093EA001092EA008091EB008860BE
:103D00008093EB001092E9008091E800877F809318
:103D1000E8000E940D1CACC08111AAC010919C0249
:103D20001F778091E3008078812B8093E30080915E
:103D3000E800877F8093E8000E940D1C8091E800D6
:103D400080FFFCCF8091E30080688093E300111135
:103D500002C082E001C083E08093990289C080584C
:103D6000823008F085C080919C0290919D028C3D2C
:103D700053E0950779F583E08A838AE289834FB718
:103D8000F894DE01139620E03EE051E2E32FF0E0EC
:103D900050935700E49120FF03C0E295EF703F5F1E
:103DA000EF708E2F90E0EA3010F0C79601C0C096F9
:103DB0008D939D932F5F243149F74FBF8091E80089
:103DC000877F8093E8006AE270E0CE0101960E944E
:103DD000191B16C060919E0270919F02AE014F5F49
:103DE0005F4F0E94731ABC01892B09F441C0909166
:103DF000E800977F9093E80089819A810E94771B61
:103E00008091E8008B778093E80032C0803881F59C
:103E10008091E800877F8093E800809195028093ED
:103E2000F1008091E8008E7772CF811121C08091DE
:103E30009C0290919D0299270297D4F48091E8000A
:103E4000877F8093E80080919C02809395020E9476
:103E50000D1C80919502811106C08091E30087FDC1
:103E600002C081E001C084E0809399020E9476192B
:103E70008091E80083FF0AC08091E800877F8093EB
:103E8000E8008091EB0080628093EB00AA960FB669
:103E9000F894DEBF0FBECDBFDF91CF911F91089583
:103EA0000895CF93809199028823A1F0C091E900F1
:103EB000CF709091EC00892F817090FD80E8C82B25
:103EC0001092E9008091E80083FD0E94F01DCF7000
:103ED000C093E900CF91089597FB072E16F4009444
:103EE00007D077FD09D00E94861F07FC05D03EF45D
:103EF000909581959F4F0895709561957F4F089596
:103F0000EE0FFF1F0590F491E02D0994AA1BBB1B37
:103F100051E107C0AA1FBB1FA617B70710F0A61BC9
:103F2000B70B881F991F5A95A9F780959095BC01EA
:103F3000CD010895FB01DC0104C08D910190801931
:103F400021F441505040C8F7881B990B0895F99906
:103F5000FECF92BD81BDF89A992780B50895A8E15A
:103F6000B0E042E050E00C94DB1F262FF999FECF21
:103F700092BD81BDF89A019700B4021639F01FBABC
:103F800020BD0FB6F894FA9AF99A0FBE08950396D9
:103F9000272F0E94B61F0E94B51F252F0E94B61F13
:103FA000242F0C94B61F0196272F0E94B61F0C9445
:103FB000B51FDC01CB01FC01F999FECF06C0F2BDB3
:103FC000E1BDF89A319600B40D9241505040B8F7D7
:063FD0000895F894FFCFF4
:103FD600C8000302280850011E0A1401B818DB188D
:103FE600BC184B194719BB1801F037923067663673
:103FF60034E200E900EA00B500B600B700CD008360
:1040060001CC008A01920194012102230224022597
:1040160002260227022A02B300B4006F0070008154
:104026008283E200E900EA00B500B600B700CD00E1
:104036008301CC008A019201940121022302240209
:104046002502260227022A02B300B4006F00700080
:0440560081828300E0
:00000001FF
